:02000000EA2AEA
:08000800FF00030E8312031335
:10001000B4000A0EB500040EB6008A110A12142BA1
:100020000330EB07EB0CEB0C7F30EB050000EB0B28
:10003000162808000000000000000000000000007A
:100040000000E60B1A28080083120313E901EA01F5
:10005000D008031D2D280230E9005008003C031889
:1000600037280A305002031837285008E900500892
:10007000093C031844280D305002031844280A3064
:100080005002E9000130EA0050080C3C03185028E7
:1000900016305002031850280C305002E900EA01D3
:1000A0005008153C03185D285008173C031C5D28B8
:1000B00016305002E9000130EA004F088500861032
:1000C0000615861106160A30EB00102006124E089F
:1000D000850086140615861106160A30EB001020DE
:1000E00006126908850086100611861506160A3064
:1000F000EB00102006126A03031981280F308500D7
:1001000083286A08850086140611861506160A30AB
:10011000EB0010200612080083120313E601E7012A
:10012000E801CC08031DB2283B304D020318A72874
:10013000CD0A4D08E600CE016608093C0318A42844
:10014000CE0A0A30E6029C286608CF00C628CD01F8
:10015000CF01CE01173050020318B028D00AC628AC
:10016000D001C6284808E800E7016808003C0318E9
:10017000BD28E8030A30E707B52847086707CD0020
:100180004708CF004808CE004608D0002420CC0104
:100190000800031083120313AF0CAE0CAD0CAC0CB3
:1001A000AF130618AF170130C10008008312031304
:1001B000DD0120305D0203180800C1080319DD28A5
:1001C000C101DD0AD92883120313DD0120305D024D
:1001D0000318F028C1080319EA28C101DD0AE6283E
:1001E000BB01BC012C082406DE002D082506DF001B
:1001F0002E082606E0002F082706E1002C08280616
:10020000E2002D082906E3002E082A06E4002F0844
:100210002B06E500B70120303702031808005E1CEA
:10022000BB0A0310E10CE00CDF0CDE0C621CBC0A04
:100230000310E50CE40CE30CE20CB70A0B29831263
:1002400003138612DD01C008031DBF08031DDD0A6C
:10025000DD08031D0800C10803192B29C101BA01DB
:100260002C082006B0002D082106B1002E08220619
:10027000B2002F082306B300B7012030370203185D
:100280004B2930184429BA0A0310B30CB20CB10C34
:10029000B00CB70A3D293D083A02031C2229BF08C9
:1002A000031D22290130BF003F03031D2229B8018D
:1002B0002030380203186229C10803195C29C101E2
:1002C000B80A5829BA012C082006DE002D0821069C
:1002D000DF002E082206E0002F082306E1005E085A
:1002E000B0005F08B1006008B2006108B300B70158
:1002F000203037020318862930187F29BA0A0310E4
:10030000B30CB20CB10CB00CB70A78293D083A0214
:10031000031C8D290130C0002229BF012229831628
:1003200003138501C13086008312850186010730E1
:100330009F00831681128111011181100110011695
:1003400083129012101690100C101010C3308F00F2
:1003500001308E0010149210121012139212121209
:1003600092111211C0308B00013083168C000800EE
:1003700083120313DB01DC018F218312C201C3014D
:10038000BF01C0011F21C4011F30B900C701C8014E
:10039000D501D601C901CA018616CB01D1010330AE
:1003A00051020318E829E3203E083B02031CDC2924
:1003B0000310C80D4814E6293E083C02031CE4293A
:1003C0000310C80D4810E6290130CB00D10ACF290F
:1003D000D620CB08031D062AD10104305102031890
:1003E000062AE3203E083B02031CFA290310C70D2E
:1003F0004714042A3E083C02031C022A0310C70DBE
:100400004710042A0130CB00D10AED29CB08031D87
:100410002B2AD101033051020318112AD620D10A08
:100420000A2AD1010230510203182B2AE3203E0888
:100430003B02031C1F2A0310D60D5614292A3E081E
:100440003C02031C272A0310D60D5610292A01301E
:10045000CB00D10A122ACB08031D492AD620D1018C
:10046000043051020318492AE3203E083B02031CD2
:100470003D2A0310D50D5514472A3E083C02031CA3
:10048000452A0310D50D5510472A0130CB00D10A5B
:10049000302ACB08031D902A4808D200D801520800
:1004A000003C0318572A0A30D807D2034F2A4708BE
:1004B0005807D900DA015608D4005408003C031844
:1004C000652A0A30DA07D4035D2A55085A07D7008F
:1004D0003B30590203186E2AD90A762AD9011730FF
:1004E00057020318752AD70A762AD701D20159086C
:1004F000093C03187F2AD20A0A30D902772A520807
:10050000C8005908C700D4015708093C03188C2AB1
:10051000D40A0A30D702842A5408D6005708D500D6
:10052000CB08031DAB2AD1012630510203189B2AA8
:10053000D620D10A942AE3203E083B02031CA32ABA
:100540000130DC00AB2A3E083C02031CA92ADC0176
:10055000AB2A0130CB00CB08031DE82AD301D1011F
:10056000560851020318B82A0A30D307D10AB02A14
:1005700055085307D300DC08031DD02A5308073C55
:10058000031CC52A10305307C6005308073C031844
:10059000D02A5308173C031CD02A08305302C60047
:1005A0005C03031DE52A5308063C031CDA2A1130BC
:1005B0005307C6005308063C0318E52A5308173CA6
:1005C000031CE52A07305302C6000130CC00C029C5
:1005D000CC01C02983120313A001A101A201FC30A8
:1005E000A300A401A501FF30A600FF30A7008030C2
:1005F000A800FF30A900FF30AA00FF30AB00AC011B
:10060000AD01AE01AF011F30BD001C30BE00C10105
:10061000C201C301C401C501CC01CD01CE01CF018E
:10062000D0018A110A12B829831203130C1C502B13
:100630000C101010C3308F0004308E001014C9202D
:100640001F3039020318262BB90A502BB9013B3051
:10065000440203182D2BC40A2F2BC4018C204408FC
:10066000C500C3014508093C03183A2BC30A0A30E8
:10067000C502322B4508C2004208850086100611CB
:10068000861106160130E6001A200612430885007E
:1006900086140611861106160130E6001A2006128D
:1006A000360E8400350E8A00340E8300FF0E7F0E56
:0206B00009003F
:02400E00E93F88
:00000001FF
